:1000000012C0189518951895189518951895189563
:100010001895189518951895189518951895189578
:100020001895189518958FE58DBFC0E4E8E34E2E1E
:1000300084E08EBFD4E0F4E05F2EEEEFF3E0A0E6C4
:10004000B0E0A89584B7082E877F84BF88E1992700
:1000500081BD91BD88278D933197E9F766248FEF95
:1000600081BB959A82E390E018D0959882E390E066
:1000700014D0969A82E390E010D0969882E390E0B4
:100080000CD0EFCFF894FFCF3197F1F70895689433
:1000900062F80895E89462F80895EF93FF93EE27CD
:1000A000E82BE92B31F0E8EEF3E03197F1F7019717
:0800B000D1F7FF91EF910895D3
:00000001FF
